:020000040000FA
:0400000000003A289A
:08000800A00003088301A10020
:100010000A08A2000408A30083160B08203903195C
:100020002B280B080439031D16282B283520A7037D
:10003000031D2928241820280130A700241429286A
:10004000A50A2410A609A60AA60A2608A7000319CD
:10005000A70A83160B1183012308840022088A0053
:1000600021088300A00E200E090083121E08A6009E
:100070009F140800FF2383169000D8308500831258
:100080008501831699018312810107309900831637
:10009000843081008B160B118B1718309F00831250
:1000A0000D309F0000000000000000009F1424108D
:1000B0000130A700A50125080339820762286628B8
:1000C0006A286E2883121F3085005B2883123D301A
:1000D00085005B2883123E3085005B2883123B300D
:0400E00085005B2814
:1006600045344C3445344334543452344F344E348E
:1006700049344334203453344534513455344534AB
:100680004E344334453452342034503449344334A6
:10069000203431343234463436343734353420342F
:1006A00042345934203444345234203452342E34B9
:1006B0002034453452344C344934433448342034A3
:1006C00063342F346F342034453449344434203477
:1006D00043344F34523450342E34203426342034B2
:1006E0004234593420344B3445344934543448343A
:1006F000203459344F3455344E34473442344C341A
:100700004F344F344434203463342F346F34203426
:1007100059344234203454344534433448342E342C
:1007200020344134553447342E342034323430347C
:1007300030343834203420342034203420342034F1
:100740002034203420342034203420342034203409
:1007500020342034203420342034203420342034F9
:100760005434483449345334203453344F344634A9
:10077000543457344134523445342034493453349A
:100780002034503452344F34563449344434453490
:10079000443420344F344E34203441344E342034E9
:1007A00041345334203449345334203443344F34A7
:1007B0004E3444344934543449344F344E342E3456
:1007C0002034203420342034203420342034203489
:1007D0002034203420342034203420342034203479
:02400E00843FED
:00000001FF
